:0400000002012132A6
:02000B002100D2
:03001300C20132F5
:01001B0032B2
:0100230032AA
:10010000C0E0C0D0D530157530C8D200D5310D75DE
:100110003114D5320775323CD203211CD0D0D0E047
:100120003275B07F7590FF75815F758C0675892279
:10013000D28CD2AFD2A97531147530FA75323CC267
:1001400000C203C201C202C204A202B392B4A2045A
:10015000B392B53000F3C20020B30AC202C204C297
:1001600001D2B7804230022CA2B282045002803702
:1001700020B23AD204D53407C201D2B7753600D5C1
:10018000332BD201C2B775360075323CC202C204AD
:10019000C203801930B210D53513D202753364759D
:1001A00034147535648006C202C20480EF20010455
:1001B000D2B72149300392C203D3E5363400F53675
:1001C0004037E590F4A2E09205A2E292E0A2E1922B
:1001D000E2A20592E1A2E49205A2E692E4A2E592EF
:1001E000E6A20592E5FF54F0C475F00AA4FEEF54B0
:1001F0000F2EFFC3E5369F4009D2B7C20175360006
:060200008002C2B7214993
